:100000006E28A4008417800484138E010C1C8E00BB
:100010000F20031969280F20031969280F282408C5
:100020008E0601308C008D01000824050E06031D8C
:1000300008008C0A03198D0F142808008F018E0008
:10004000FF308E07031C8F07031C692803308D00C7
:10005000DF302C2020288D01E83E8C008D09FC30FB
:10006000031C35288C07031832288C0764008D0F79
:1000700032280C183B288C1C3F2800003F28080021
:100080008E000330432894000F080D02031D4A28F8
:100090000E080C0204300318013003190230140555
:1000A000031DFF306928103094008D018C01930CE2
:1000B000920C031C61280E088C070F0803180F0F01
:1000C0008D078D0C8C0C910C900C940B57281008FC
:1000D0006928831303138312640008008316083011
:1000E00085008601831285018601DF2801308C009E
:1000F00005308400083001200C08AA000D08AB0070
:100100002A088C002B088D008F0150304020031DE1
:100110008B28AD0108002A088C002B088D008F0168
:1001200075304020031D97280130AD0008002A08D3
:100130008C002B088D008F018E304020031DA328DA
:100140000230AD0008002A088C002B088D008F01BA
:10015000A2304020031DAF280330AD0008002A085C
:100160008C002B088D008F01BB304020031DBB2865
:100170000430AD0008000530AD00080015308600E1
:1001800032301E20B030860032301E2015308600FE
:1001900032301E20B030860064301E200E308600C3
:1001A00032301E20C830860032301E200E308600CD
:1001B00032301E20C83086005F301E2008008501C6
:1001C00086010130A800A9010130AC0064000930AB
:1001D0002C020318F628280886000310A80DA90D84
:1001E00003308F00E8301F20AC0FE6288601762010
:1001F0002D088D00053C031C15298D0D05218C0053
:100200000D1005218A000C08820001308A000D08BB
:1002100082070134BB34013460340134B634013414
:1002200016340134B63401346034F7280130AC00A0
:10023000640004302C0203182729E730860032308E
:100240001E20E330860032301E20AC0F18297620A5
:1002500064002D08033C031DF7280130AC00640046
:1002600010302C0203184029E73086007620640005
:100270002D08033C031DF728C8301E20AC0F2F2982
:100280009F30860001308F0090301F20873086001D
:1002900001308F0090301F20762064002D08033C31
:1002A000031D53294029BE20762064002D08013CFF
:1002B0000319F72864002D08053C0319F728532972
:1002C0000130AC0064001A302C0203187D29E330A1
:1002D000860064301E20762064002D08023C03193D
:1002E0008E2964002D08043C03198E2964002D0812
:1002F000033C03191629AC0F62290130AC006400DD
:1003000008302C0203188E298030860032301E20DF
:10031000E330860032301E20AC0F7F297620640047
:100320002D08023C0319A42964002D08043C03197C
:10033000A42964002D08033C0319162964002D0824
:10034000003C0319BB298E290130AC006400043045
:100350002C020318B529E330860050301E20E73008
:10036000860050301E20AC0FA629F728E330860007
:1003700064301E20F7280130AC00640009302C02E4
:100380000318D029FF30860001308F0090301F20E5
:10039000E730860001308F0090301F20AC0FBD2960
:1003A000762064002D08003C031DF72813308F00D1
:1003B00088301F20762064002D08003C031DF7289C
:1003C0000130AC0064000B302C020318F12980309E
:1003D000860050301E20E330860050301E20AC0FC7
:1003E000E229762064002D08003C031DF7280B301D
:1003F0008F00B8301F200130AC00640015302C0293
:100400000318052ABE20AC0FFD29762064002D08B4
:0C041000003C031DF728BB2963000C2AE8
:02400E00FE3F73
:00000001FF
